:020000040800F2
:10000000600900204501000819110008811000084E
:1000100015110008B10100082F3100080000000090
:10002000000000000000000000000000F1270008B0
:10003000110E000800000000912300083D2A00086E
:100040005F0100085F0100085F0100085F01000810
:100050005F0100085F0100085F0100085F01000800
:100060005F0100085F0100085F0100085F010008F0
:100070005F0100085F0100085F0100085F010008E0
:100080005F0100085F0100085F0100085F010008D0
:100090005F0100085F0100085F0100085F010008C0
:1000A0005F0100085F0100085F0100085F010008B0
:1000B0005F010008A52A00085F0100085F01000831
:1000C0005F0100085F0100085F0100085F01000890
:1000D0005F010008852C0008E12C0008C52D0008F0
:1000E0005F0100085F0100085F0100085F01000870
:1000F0005F0100085F0100085F0100085F01000860
:100100005F0100085F0100085F0100085F0100084F
:100110005F0100085F0100085F0100085F0100083F
:100120005F0100085F0100085F0100085F0100082F
:10013000DFF80CD000F02AF80048004735320008FC
:10014000600900200648804706480047FEE7FEE7B2
:10015000FEE7FEE7FEE7FEE7FEE7FEE7FEE7FEE777
:10016000412A000831010008D2B201E000F8012B59
:10017000491EFBD270470022F6E710B513460A4627
:1001800004461946FFF7F0FF204610BD064C074D08
:1001900006E0E06840F0010394E807009847103457
:1001A000AC42F6D3FFF7C8FFF03500081036000860
:1001B00000BFFEE710B502460B460020002104E018
:1001C000545C0444E0B24C1CE1B29942F8DBC443F5
:1001D000E0B2441CE0B210BDFEB5002000900190DA
:1001E000029000F067FF3A4800780A2822D1394887
:1001F000007839490978884218D13648407836491C
:100200004978884212D13348007A3349097A8842C2
:100210000CD13048407A3049497A884206D12F487B
:10022000008840F400402D49088003E0142129484B
:10023000FFF7A1FF2948008800F40040002846D0BD
:10024000274800210160017126480160017126489C
:100250000160017125480160017100202149087089
:100260001C48007948701B4840798870194880798B
:10027000C8701848C079087100201D4908701948D5
:10028000407848701748807888701648C078C870E1
:1002900014480079087113484078040611488078A2
:1002A00005041048C0780602601930440D490979E8
:1002B000471801200F49087000F0FCFE0020044997
:1002C00008700649088014210248FFF754FFFEBD5C
:1002D00009000020D40100200C0000200A000020AA
:1002E00034000020160000203C00002041000020C7
:1002F0001B0000204900002010B588B07F4800781E
:10030000012838D100207D490870FC207C49087004
:10031000112048707B48007888707A484078C8700F
:100320007848807808717748C078487175480079B6
:10033000887107217248FFF73DFF7149C87100209D
:1003400071490860FF22E121012001F06FFF0823BD
:100350006B4AA821012001F02BFF012001F058FA7F
:1003600001206A49C1F8A40169490870002069495F
:10037000088000F09FFE6748008840F6B831884248
:100380007BDC00F097FE604884380068002857D175
:1003900000F090FE6946012001F0E8FE0446204688
:1003A00002F074FA5CA002F07BFA04F040004028EE
:1003B000EDD100208DF80A000721684600F029FDE4
:1003C00055A002F06DFA9DF801004E490978884267
:1003D00054D19DF802004B49497888424ED19DF88E
:1003E000030048498978884248D19DF8040045496E
:1003F000C978884242D19DF805004249097988426E
:100400003CD14348007801281BD141480078401C6A
:100410003F49087012203A49487007213848FFF7D1
:10042000C9FE3749C8710020374908600823344A9B
:10043000A821012001F0BCFE01203449C1F8A4012B
:1004400058E00020324908700E21344800F0E1FCE9
:1004500031A002F025FA32480178012001F032FA89
:1004600010202E4948700E212C4802F003FA2DA0CE
:1004700002F016FA012008B010BD16E00020224953
:10048000086011201E49487007211D48FFF792FEA1
:100490001B49C87108230A46A821012001F088FEE3
:1004A00001201A49C1F8A40124E000201549087070
:1004B00048708870C87008711B490870487088704F
:1004C000C87008711949087048708870C870087140
:1004D0001749087048708870C870087130200F493B
:1004E00048700E210D4802F0C5F912A002F0D8F9AB
:1004F0000120C0E700F0DEFD0020BCE74600002040
:100500004A00002034000020A481214200802142C2
:100510008A000020260000200A000000C8030020F6
:10052000320000204F4B0A00410000201B00002039
:1005300016000020333030300A00000010B588B0BB
:100540005648008840F6B831884271DA544800684D
:1005500000286ED100F0AEFD6946012001F006FED4
:10056000044604F040004028F3D100208DF80A0032
:100570009DF8010078B99DF8020060B99DF803006C
:1005800048B900204749087048708870C8700871E1
:10059000012008B010BD44480078072803D0424825
:1005A00000780D280FD100203E4908709DF800000A
:1005B00048709DF8010088709DF80200C8709DF891
:1005C0000300087159E038480078082810D19DF8D8
:1005D0000100344908709DF8020048709DF803003E
:1005E00088709DF80400C8709DF80500087144E00B
:1005F0002D480078092803D02B4800780E2819D1FF
:100600000020284908709DF8010080F053004870D0
:100610009DF8020080F0430088709DF8030080F090
:100620004400C8709DF8040080F05800087124E070
:1006300028E024E01C48007814280FD10020194934
:1006400008709DF8040048709DF8050088709DF8BA
:100650000600C8709DF8070008710EE000201149DF
:1006600008709DF8010048709DF8020088709DF8A0
:100670000300C8709DF804000871012089E700F0AC
:1006800019FD08E000200749087048708870C8709C
:10069000087101207DE700207BE700003A00002080
:1006A00020812142410000203200002010B500F0DE
:1006B00001FDFE480078082829D1FD4800787528FA
:1006C00025D1FB484078702821D1F94880786428EA
:1006D0001DD1F748C078612819D1F54800797428F0
:1006E00015D1F3484079652811D10020EF490870F1
:1006F00000BFF048006800F4E060EF490843001DC7
:10070000EC490860BFF34F8F00BF00BFFEE7E84829
:100710000078752807D0E6480078FA2803D0002032
:10072000E249087010BDE14800780E2800DAF9E7C8
:10073000DE480078401EDE49085CFB2800D0F1E767
:10074000DB48807AA02804D1D8480078152800D04A
:10075000E8E7D64800780E281ED1D5480078FA2858
:1007600014D1D348407BFB2810D1D448008840F4F2
:100770000040D24908800020CC4908700E21CC48A6
:1007800000F047FBCEA002F08BF84AE00020C749FA
:100790000870CA49088044E0C448007815281ED172
:1007A000C3480078FA2814D1C148007DFB2810D135
:1007B000C248008840F40040C04908800020BB497E
:1007C00008701521BA4800F024FBBDA002F068F8BB
:1007D00027E00020B5490870B849088021E0B348F7
:1007E000007811281DD1B2480078FA2814D1B048F9
:1007F000007CFB2810D1B148008840F40040AF498C
:1008000008800020A94908701121A94800F001FBC7
:10081000ABA002F045F804E00020A4490870A74905
:100820000880A648008800F40040002871D000F03D
:1008300041FC9F488079A34988719D48C179A148AE
:10084000C1719B48017A9F4801729948417A9D483D
:1008500041729748807A9B498872084680799A4904
:1008600088719848C1799848C1719648017A96482C
:1008700001729448417A944841729248807A94284F
:100880004CD018DC732834D00CDC252825D004DCAF
:1008900021281AD022287DD11BE0262821D07128BA
:1008A000F9D122E0742828D075282AD078282CD0B5
:1008B0008228F0D12EE0A03809286BD2DFE800F0C2
:1008C000329CA0F5F4F3F2F1F00000207D4988722B
:1008D000DAE100207B498872D6E1002079498872EC
:1008E000D2E1002077498872CEE1002075498872F4
:1008F000CAE1002073498872C6E1002071498872FC
:10090000C2E100206F498872BEE100206D49887203
:10091000BAE1BDE100206B498872B5E10020694968
:100920008872B1E1002061490870664880796749A2
:1009300088716448C1796548C1716248017A634829
:1009400001726048417A614841725E48807A5F492D
:1009500088725748407B5B4948735548817B5948AA
:1009600081735348C17B5748C1735148017C554836
:1009700001744F48417C534841744D48407B544971
:1009800008704B48807B48704948C07B8870484855
:10099000007C00E077E1C8704548407C0871012088
:1009A0004C49087000204C490880012000F030FFBD
:1009B0004AA001F075FF04E0FFF79EFC044604B175
:1009C00000E0F9E700BF45A001F06AFF00204549BB
:1009D000087048708870C870087143490870487082
:1009E0008870C87008714149087048708870C87074
:1009F00008713449887247E100203249887243E126
:100A00003B48007830B9384800210160017101206D
:100A1000374908703448407848B93348807830B94D
:100A20003148C07818B93048007900B92CE100206D
:100A30001E490870234880792E4988712148C17960
:100A40002C48C1711F48017A2A4801721D48417A19
:100A5000284841721B48807A264988720120C87252
:100A600006200873002048731F48017821488173CD
:100A70001D4841781F48C1731B4881781D48017487
:100A80001948C1781B484174174801791948817485
:100A9000162101F0EFFE322002F078FB16212BE048
:100AA000A8E0ECE0E7E0E2E03AE038E00300002014
:100AB0000C0100200CED00E00000FA05040000200D
:100AC0000A000000000300209C020020C803002050
:100AD0003400002046000020260000203030303056
:100AE0000A000000410000201B000020160000202A
:100AF0002B00002064030020664800F08AF9AFF262
:100B0000400001F0CDFE00206349087048708870F5
:100B1000C87008716149087061498872B4E0B3E037
:100B200000206049087060480178012000F0CAFE8A
:100B300000205E4908805EA001F0B2FE04E0FFF7ED
:100B4000FDFC044604B100E0F9E700BF58A001F045
:100B5000A7FE534880794F4988715148C1794D4863
:100B6000C1714F48017A4B4801724D48417A49485A
:100B700041724B48807A474988720120C87206202A
:100B80000873002048734C480178424881734A48F2
:100B900041784048C173484881783E4801744648CE
:100BA000C1783C484174444801793A48817416211F
:100BB00001F060FE322002F0E9FA1621354800F01B
:100BC00028F93CA001F06CFE00203B4908704870F9
:100BD0008870C87008713049087048708870C87093
:100BE00008713649087048708870C87008712C49BF
:100BF000887249E03248407B2B4908702848807948
:100C0000304988712648C1792E48C1712448017A3B
:100C10002C4801722248417A2A4841722048807A41
:100C200028498872012048700E21264801F022FED2
:100C3000322002F0ABFA1C4800782349088001F00A
:100C4000E1FD00201C49087048708870C870087168
:100C50001149087048708870C87008711749087089
:100C600048708870C87008710D4988720CE00020C7
:100C70000B49887208E000200949887204E00020CE
:100C80000749887200E000BF00BF00200F490880BC
:100C900000BF47E5640300201B0000202B0000205C
:100CA0000003002003000020320000203A00002052
:100CB000343434340A0000004100002016000020C3
:100CC0000C0100202C04002034050020040000202A
:100CD000FA204A49087010204870002088700021CE
:100CE0004648C1700171417100204449887100215A
:100CF0004248C1710172417200204049C87400210C
:100D00003E480175FB203D494875FA203C49087072
:100D1000102048700020887000213948C17001718E
:100D2000417100203649887100213548C171017236
:100D300041720020324981F84B000021304880F890
:100D40004C10FB202E4981F84D00FA202D490870E7
:100D5000102048700020887000212A48C17001715D
:100D6000417100202749887100212648C171017214
:100D7000417200202349C872002122480173FB20E0
:100D800020494873FA20204908701020487000203C
:100D9000887000211C48C1700171417100201A49FE
:100DA000887100211848C1710172417200201649F2
:100DB000C874002114480175FB2013494875FA20B6
:100DC00012490870102048700020887000210F48D8
:100DD000C1700171417100200C49887100210B48DC
:100DE000C1710172417200200849C8720021074890
:100DF0000173FB2005494873704700009C020020E6
:100E0000000300202C04002064030020C8030020FD
:100E100070472DE9F04104460E460DE02578281173
:100E200000F030F9074601F031FD284600F02AF9BC
:100E3000074601F02BFD641C301EA6F10101CEB265
:100E4000ECD1BDE8F081000030B5044604254FF434
:100E5000302000F06FF80546042D17D10C480069CA
:100E600040F002000A49086108464461006940F008
:100E7000400008614FF4302000F05CF8054604485B
:100E8000006941F6FD71084001490861284630BDFE
:100E90000020024004200B49C96801F0010109B19A
:100EA00001200EE00749C96801F0040109B10220E0
:100EB00007E00449C96801F0100109B1032000E00E
:100EC00004207047002002400348006940F0800081
:100ED00001490861704700000020024070B50446D7
:100EE0000D460426F00200F025F80646042E11D126
:100EF0000948006940F00100074908612580F002B7
:100F000000F018F806460448006941F6FE710840F2
:100F100001490861304670BD002002400248034983
:100F2000486003484860704723016745002002403D
:100F3000AB89EFCD00B502460423FFF7ABFF0346B4
:100F400003E0FFF7A7FF0346521E012B01D1002A41
:100F5000F7D102B90523184600BD2DE9F04102463C
:100F600000250026002000230024002791F803C05C
:100F70000CF00F0591F803C00CF0100CBCF1000F41
:100F800003D091F802C04CEA050591F800C0BCF10D
:100F9000000F31D0146800202BE04FF0010C0CFA48
:100FA00000F3B1F800C00CEA03069E4220D1830092
:100FB0004FF00F0C0CFA03F7BC4305FA03FC4CEAA4
:100FC000040491F803C0BCF1280F06D14FF0010CC6
:100FD0000CFA00FCC2F814C00AE091F803C0BCF19E
:100FE000480F05D14FF0010C0CFA00FCC2F810C0FC
:100FF000401C0828D1D31460B1F800C0BCF1FF0F29
:1010000034DD546800202EE000F1080C4FF0010898
:1010100008FA0CF3B1F800C00CEA03069E4221D195
:1010200083004FF00F0C0CFA03F7BC4305FA03FCE6
:101030004CEA040491F803C0BCF1280F05D100F17B
:10104000080C08FA0CF8C2F8148091F803C0BCF13F
:10105000480F07D100F1080C4FF0010808FA0CF80E
:10106000C2F81080401C0828CED35460BDE8F0813F
:10107000416170470161704701460A8890B270472C
:1010800000BFFEE70146002001F00F02092A04DC40
:1010900001F00F0202F1300003E001F00F023732DD
:1010A000D0B270474CF6CC40014908607047000050
:1010B0000030004010B500F013F810BD70B50546C3
:1010C0000C4645F2555000F01FF8284600F010F885
:1010D000204600F013F800F003F8FFF7E3FF70BDBF
:1010E0004AF6AA200149086070470000003000401D
:1010F00001494860704700000030004001498860A5
:10110000704700000030004001490860704700004F
:101110000030004000BFFEE7704700007CB5054688
:1011200012A103C9CDE900010821284601F038FBCE
:1011300005236A463021284601F03AF805236A461D
:101140001021284600F0A4FF002406E01DF804004A
:10115000A52800D003E0601CC4B2052CF6DB00BF5C
:10116000052C01D001207CBD0020FCE7A5A5A5A58C
:10117000A500000008B501211C2001F01BF940204A
:10118000ADF8000010208DF8030003208DF8020058
:1011900069463248FFF7E1FE40213048FFF76AFF19
:1011A0001020ADF8000069462D48FFF7D6FE10214B
:1011B0002B48FFF75FFF8020ADF8000048208DF836
:1011C000030003208DF8020069462448FFF7C5FE9E
:1011D0004FF40070ADF8000010208DF803000320DC
:1011E0008DF8020069461D48FFF7B7FE4FF4007105
:1011F0001A48FFF73FFF4FF48050ADF800006946F2
:101200001648FFF7AAFE4FF480511448FFF732FF4B
:101210004FF48070ADF8000048208DF803000320E3
:101220008DF8020069460D48FFF797FE01F0E6F9D8
:1012300001F0A2F900200B49086001200A49C1F819
:101240009001002007490C31086001200749C1F8CE
:10125000B0010821002001F0A3FA08BD000C0140F4
:101260000008014098812142000021420080214273
:1012700010B5044602222321204600F0D7FF0423A4
:101280001E4A2A21204600F093FF04231B4A3021E6
:10129000204600F08DFF3F222121204600F0C6FFAE
:1012A0003F222221204600F0C1FF1C22252120469A
:1012B00000F0BCFF04222621204600F0B7FF0F22D9
:1012C0002021204600F0B2FF0A223121204600F002
:1012D000ADFF01223D21204600F0A8FF00223C2165
:1012E000204600F0A3FF70222721204600F09EFF39
:1012F000FF22E221204600F099FF10BDEA350008E8
:1013000010B5044602222321204600F08FFF05235A
:101310001E4A2A21204600F04BFF05231B4A30219C
:10132000204600F045FF3F222121204600F07EFFAD
:1013300001222221204600F079FF1A222521204691
:1013400000F074FF24222621204600F06FFF0F22B8
:101350002021204600F06AFF0A223121204600F0B9
:1013600065FF01223D21204600F060FF00223C2164
:10137000204600F05BFF70222721204600F056FF38
:10138000FF22E221204600F051FF10BD95350008F4
:1013900010B5044602222321204600F047FF042313
:1013A0001E4A2A21204600F003FF04231B4A302155
:1013B000204600F0FDFE30222121204600F036FFBD
:1013C00001222221204600F031FF12222521204651
:1013D00000F02CFF24222621204600F027FF0F22B8
:1013E0002021204600F022FF08223121204600F073
:1013F0001DFF01223D21204600F018FF00223C2164
:10140000204600F013FF70222721204600F00EFF37
:10141000FF22E221204600F009FF10BDCC35000874
:1014200010B5044602222321204600F0FFFE0423CB
:101430001E4A2A21204600F0BBFE04231B4A30210D
:10144000204600F0B5FE30222121204600F0EEFEBD
:1014500001222221204600F0E9FE332225212046E8
:1014600000F0E4FE07222621204600F0DFFE0F22D6
:101470002021204600F0DAFE05223121204600F02E
:10148000D5FE01223D21204600F0D0FE00223C2165
:10149000204600F0CBFE70222721204600F0C6FE39
:1014A000FF22E221204600F0C1FE10BDE535000814
:1014B00010B5044602222321204600F0B7FE042383
:1014C0001E4A2A21204600F073FE04231B4A3021C5
:1014D000204600F06DFE30222121204600F0A6FEBD
:1014E00001222221204600F0A1FE282225212046AB
:1014F00000F09CFE0C222621204600F097FE0F22D1
:101500002021204600F092FE06223121204600F0E4
:101510008DFE01223D21204600F088FE00223C2164
:10152000204600F083FE70222721204600F07EFE38
:10153000FF22E221204600F079FE10BDC2350008EE
:1015400010B5044602222321204600F06FFE04233A
:101550001E4A2A21204600F02BFE04231B4A30217C
:10156000204600F025FE30222121204600F05EFEBC
:1015700001222221204600F059FE16222521204674
:1015800000F054FE04222621204600F04FFE0F22D8
:101590002021204600F04AFE08223121204600F09A
:1015A00045FE01223D21204600F040FE00223C2164
:1015B000204600F03BFE70222721204600F036FE38
:1015C000FF22E221204600F031FE10BDDB3500088D
:1015D00010B5044602222321204600F027FE0423F2
:1015E0001E4A2A21204600F0E3FD04231B4A302135
:1015F000204600F0DDFD30222121204600F016FEBD
:1016000001222221204600F011FE3322252120460E
:1016100000F00CFE04222621204600F007FE0F22D7
:101620002021204600F002FE09223121204600F050
:10163000FDFD01223D21204600F0F8FD00223C2165
:10164000204600F0F3FD70222721204600F0EEFD39
:10165000FF22E221204600F0E9FD10BDB835000868
:1016600010B5044602222321204600F0DFFD0523A9
:101670001E4A2A21204600F09BFD05231B4A3021EB
:10168000204600F095FD3F222121204600F0CEFDAE
:1016900001222221204600F0C9FD122225212046E8
:1016A00000F0C4FD04222621204600F0BFFD0F22D9
:1016B0002021204600F0BAFD0A223121204600F008
:1016C000B5FD01223D21204600F0B0FD00223C2165
:1016D000204600F0ABFD70222721204600F0A6FD39
:1016E000FF22E221204600F0A1FD10BD8635000852
:1016F00010B5044602222321204600F097FD052361
:101700001E4A2A21204600F053FD05231B4A3021A2
:10171000204600F04DFD30222121204600F086FDBC
:1017200001222221204600F081FD1222252120469F
:1017300000F07CFD21222621204600F077FD0F22BB
:101740002021204600F072FD0A223121204600F0BF
:101750006DFD00223D21204600F068FD01223C2164
:10176000204600F063FD70222721204600F05EFD38
:10177000FF22E221204600F059FD10BD7735000818
:1017800010B5044601222321204600F04FFD052319
:101790001E4A2A21204600F00BFD05231B4A30215A
:1017A000204600F005FD30222121204600F03EFDBC
:1017B00001222221204600F039FD19222521204650
:1017C00000F034FD04222621204600F02FFD0F22D8
:1017D0002021204600F02AFD06223121204600F07B
:1017E00025FD01223D21204600F020FD00223C2164
:1017F000204600F01BFD70222721204600F016FD38
:10180000FF22E221204600F011FD10BDA4350008A2
:1018100010B504461CB900202749086003E00020E9
:1018200025490C31086001222321204600F0FEFCEE
:101830000323224A2A21204600F0BAFC0323204A2F
:101840003021204600F0B4FC01222121204600F086
:10185000EDFC01222221204600F0E8FC2A2225216D
:10186000204600F0E3FC04222621204600F0DEFCA6
:101870000F222021204600F0D9FC06223D212046DF
:1018800000F0D4FC01223C21204600F0CFFC702265
:101890002721204600F0CAFCFF22E221204600F06A
:1018A000C5FC1CB901200449086003E0012002497D
:1018B0000C31086010BD0000988121426D35000890
:1018C0006835000870B504460D461CB900203F4934
:1018D000086003E000203D490C310860172D69D2F3
:1018E000DFE805F00C1014181C2024282C303438A4
:1018F0003C4044484C5054585C6064002046FFF71C
:10190000F7FE57E0204600F0A3FA53E0204600F02F
:1019100077FB4FE02046FFF7A3FE4BE0204600F0A8
:1019200007FA47E0204600F0E3F843E02046FFF7DF
:10193000E7FC3FE0204600F0B3F93BE0204600F032
:10194000CFFA37E02046FFF71BFF33E0204600F0D8
:101950003FF82FE0204600F033FA2BE0204600F05D
:101960007FF827E02046FFF733FE23E02046FFF70D
:1019700007FF1FE02046FFF79BFD1BE0204600F01D
:1019800047F917E02046FFF703FD13E0204600F07B
:10199000F7F80FE02046FFF7D3FD0BE0204600F0FC
:1019A000E7FA07E02046FFF73BFD03E02046FFF79C
:1019B0005FFC00BF00BF1CB901200449086003E0C0
:1019C000012002490C31086070BD0000988121425D
:1019D00010B5044602222321204600F027FC0423F0
:1019E0001E4A2A21204600F0E3FB04231B4A302133
:1019F000204600F0DDFB30222121204600F016FCBD
:101A000001222221204600F011FC2022252120461F
:101A100000F00CFC20222621204600F007FC0F22BB
:101A20002021204600F002FC08223121204600F04F
:101A3000FDFB01223D21204600F0F8FB00223C2165
:101A4000204600F0F3FB70222721204600F0EEFB39
:101A5000FF22E221204600F0E9FB10BDA935000875
:101A600010B5044602222321204600F0DFFB0423A8
:101A70001E4A2A21204600F09BFB04231B4A3021EA
:101A8000204600F095FB30222121204600F0CEFBBD
:101A900001222221204600F0C9FB122225212046E6
:101AA00000F0C4FB24222621204600F0BFFB0F22B9
:101AB0002021204600F0BAFB0A223121204600F006
:101AC000B5FB01223D21204600F0B0FB00223C2165
:101AD000204600F0ABFB70222721204600F0A6FB39
:101AE000FF22E221204600F0A1FB10BDB335000823
:101AF00010B5044602222321204600F097FB05235F
:101B00001E4A2A21204600F053FB05231B4A3021A0
:101B1000204600F04DFB30222121204600F086FBBC
:101B200001222221204600F081FB1222252120469D
:101B300000F07CFB24222621204600F077FB0F22B8
:101B40002021204600F072FB0A223121204600F0BD
:101B50006DFB01223D21204600F068FB00223C2164
:101B6000204600F063FB70222721204600F05EFB38
:101B7000FF22E221204600F059FB10BD90350008FD
:101B800010B5044602222321204600F04FFB042317
:101B90001E4A2A21204600F00BFB04231B4A302159
:101BA000204600F005FB30222121204600F03EFBBC
:101BB00001222221204600F039FB14222521204653
:101BC00000F034FB04222621204600F02FFB0F22D8
:101BD0002021204600F02AFB0A223121204600F075
:101BE00025FB01223D21204600F020FB00223C2164
:101BF000204600F01BFB70222721204600F016FB38
:101C0000FF22E221204600F011FB10BDD135000873
:101C100010B5044602222321204600F007FB0423CE
:101C20001E4A2A21204600F0C3FA04231B4A302111
:101C3000204600F0BDFA30222121204600F0F6FABD
:101C400001222221204600F0F1FA1222252120460D
:101C500000F0ECFA24222621204600F0E7FA0F22B9
:101C60002021204600F0E2FA08223121204600F02F
:101C7000DDFA01223D21204600F0D8FA00223C2165
:101C8000204600F0D3FA70222721204600F0CEFA39
:101C9000FF22E221204600F0C9FA10BDC735000836
:101CA00010B5044601222321204600F0BFFA052387
:101CB0001E4A2A21204600F07BFA05231B4A3021C8
:101CC000204600F075FA30222121204600F0AEFABD
:101CD00001222221204600F0A9FA102225212046C7
:101CE00000F0A4FA04222621204600F09FFA0F22D9
:101CF0002021204600F09AFA06223121204600F0E9
:101D000095FA01223D21204600F090FA00223C2164
:101D1000204600F08BFA70222721204600F086FA38
:101D2000FF22E221204600F081FA10BD9A3500081A
:101D300010B5044602222321204600F077FA05233D
:101D40001E4A2A21204600F033FA05231B4A30217F
:101D5000204600F02DFA30222121204600F066FABC
:101D600001222221204600F061FA1222252120467C
:101D700000F05CFA24222621204600F057FA0F22B8
:101D80002021204600F052FA08223121204600F09E
:101D90004DFA01223D21204600F048FA00223C2164
:101DA000204600F043FA70222721204600F03EFA38
:101DB000FF22E221204600F039FA10BD8B350008E1
:101DC00010B5044602222321204600F02FFA0423F6
:101DD0001E4A2A21204600F0EBF904231B4A302139
:101DE000204600F0E5F930222121204600F01EFABD
:101DF00001222221204600F019FA1C22252120462A
:101E000000F014FA24222621204600F00FFA0F22B7
:101E10002021204600F00AFA08223121204600F055
:101E200005FA01223D21204600F000FA00223C2163
:101E3000204600F0FBF970222721204600F0F6F939
:101E4000FF22E221204600F0F1F910BDAE35000876
:101E500010B5044603222321204600F0E7F90523AC
:101E60001E4A2A21204600F0A3F905231B4A3021EF
:101E7000204600F09DF93F222121204600F0D6F9AE
:101E80003F222221204600F0D1F928222521204698
:101E900000F0CCF904222621204600F0C7F90B22DD
:101EA0002021204600F0C2F90A223121204600F00C
:101EB000BDF901223D21204600F0B8F900223C2165
:101EC000204600F0B3F970222721204600F0AEF939
:101ED000FF22E221204600F0A9F910BD7C35000860
:101EE00010B5044601222321204600F09FF9032368
:101EF0001E4A2A21204600F05BF903231B4A3021A9
:101F0000204600F055F930222121204600F08EF9BC
:101F100001222221204600F089F92A22252120468B
:101F200000F084F904222621204600F07FF90F22D8
:101F30002021204600F07AF907223121204600F0C6
:101F400075F900223D21204600F070F901223C2164
:101F5000204600F06BF970222721204600F066F938
:101F6000FF22E221204600F061F910BD9F350008F4
:101F700010B5044601222321204600F057F903231F
:101F80001E4A2A21204600F013F903231B4A302160
:101F9000204600F00DF930222121204600F046F9BC
:101FA00001222221204600F041F93222252120463B
:101FB00000F03CF904222621204600F037F90F22D8
:101FC0002021204600F032F910223121204600F075
:101FD0002DF901223D21204600F028F900223C2164
:101FE000204600F023F970222721204600F01EF938
:101FF000FF22E221204600F019F910BDE03500086B
:1020000010B5044603222321204600F00FF90523D2
:102010001E4A2A21204600F0CBF805231B4A302116
:10202000204600F0C5F830222121204600F0FEF8BD
:1020300001222221204600F0F9F810222521204615
:1020400000F0F4F804222621204600F0EFF80F22D9
:102050002021204600F0EAF80A223121204600F033
:10206000E5F801223D21204600F0E0F800223C2165
:10207000204600F0DBF870222721204600F0D6F839
:10208000FF22E221204600F0D1F810BD8135000882
:102090002DE9F0478046894615461E46B8F1000FE7
:1020A00016D10020174908604946404600F024FB3D
:1020B0000746002406E0FF21404600F01DFB28559E
:1020C000601CC4B2B442F6DB01200E49086015E082
:1020D00000200D4908604946404600F00DFB0746C8
:1020E000002406E0FF21404600F006FB2855601C56
:1020F000C4B2B442F6DB0120034908603846BDE8AB
:10210000F087000090012142B081214270B5054660
:102110000E4685B90020114908603146284600F076
:10212000EBFAFF21284600F0E7FA044601200C49AB
:10213000C1F890010FE000200A49086031462846A6
:1021400000F0DAFAFF21284600F0D6FA0446012012
:102150000549C1F8B001204670BD00009001214240
:1021600000002142B08121420080214270B5064624
:102170000D461021304600F013FB07213046FFF7D3
:10218000C5FF044622462721304600F04FF804F0F0
:10219000400050B10A232A4661213046FFF778FFFC
:1021A000FF22E221304600F041F8204670BD0000D9
:1021B0002DE9F0478046894615461E46B8F1000FC6
:1021C00016D10020174908604946404600F094FAAD
:1021D0000746002406E015F8011B404600F08CFA83
:1021E000601CC4B2B442F6DB01200E49086015E061
:1021F00000200D4908604946404600F07DFA074638
:10220000002406E015F8011B404600F075FA601C3A
:10221000C4B2B442F6DB0120034908603846BDE889
:10222000F087000090012142B08121422DE9F04168
:1022300004460E46154684B900201149086031460F
:10224000204600F059FA07462946204600F054FA85
:1022500001200C49C1F890010FE000200A490860F4
:102260003146204600F048FA07462946204600F04D
:1022700043FA01200549C1F8B0013846BDE8F081B4
:102280009001214200002142B08121420080214280
:1022900008B54FF4C06000F071F826208DF80000FA
:1022A00001208DF8010002208DF8020001208DF838
:1022B0000300684600F02AF827208DF8000001206E
:1022C0008DF801008DF802008DF80300684600F0DB
:1022D0001DF825208DF8000000208DF80100012058
:1022E0008DF802008DF80300684600F00FF81D20FD
:1022F0008DF8000000208DF801008DF8020001200B
:102300008DF80300684600F001F808BD70B50021A3
:1023100000230F22C47804B3154C246804F4E0644D
:10232000C4F5E064210AC1F10403CA40447804FA08
:1023300003F184781440214309010E4C0678A1551D
:10234000047804F01F050124AC4005786D11AD0040
:1023500005F1E025C5F8004109E0047804F01F0507
:102360000124AC40044D0678761145F8264070BD36
:102370000CED00E000E400E080E100E002490143F0
:10238000024A1160704700000000FA050CED00E001
:102390007047000029B1064AD2690243044BDA6152
:1023A00004E0034AD2698243014BDA6170470000BE
:1023B0000010024029B1064A92690243044B9A6117
:1023C00004E0034A92698243014B9A61704700001E
:1023D0000010024070B5012144F20D00FFF7EAFF42
:1023E00001210220FFF7D6FF042000F013FB124961
:1023F000B1F1807F00D31DE021F07F40401E4FF0FF
:10240000E022506150170F22002807DA13071D0E33
:102410000A4B00F00F04241F1D5503E013071C0E88
:10242000074B1C5400BF00204FF0E02290610720B2
:10243000106100BF70BD000080A9030018ED00E02E
:1024400000E400E070B500210023002400220025F4
:102450002C4E766806F00C0121B1042905D008291C
:1024600021D105E0284E066020E0274E06601DE0E1
:10247000244E766806F47013224E766806F4803493
:10248000022606EB93431CB9204E5E43066009E02A
:102490001C4E7668C6F34046751C1B4EB6FBF5F61F
:1024A0005E43066002E0184E066000BF00BF154E96
:1024B000766806F0F0010909154E725C0668D64090
:1024C0004660104E766806F4E061090A104E725CB0
:1024D0004668D64086600B4E766806F46051C90A9D
:1024E0000B4E725C4668D640C660064E766806F4AF
:1024F0004041890B074E725CC668B6FBF2F6066176
:1025000070BD00000010024000127A0000093D007A
:1025100090000020A000002010B586B000241421F7
:1025200001A8FDF728FE0A2201A9084800F012F8C8
:1025300000BF07E001A810F81400054A02F81400D3
:10254000601CC4B20A2CF5DB06B010BD0000030805
:102550004805002070B504460D461646002300BF0E
:1025600007E02046FEF788FD25F81300A41C581C40
:10257000C3B2B342F5DB70BD00B587B0012141F2B3
:102580000500FFF717FFE020ADF8180018208DF8C0
:102590001B0003208DF81A0006A91648FEF7DDFC83
:1025A000E0211448FEF766FD0020ADF804004FF46A
:1025B0008270ADF806000020ADF80800ADF80A0002
:1025C000ADF80C004FF40070ADF80E001820ADF817
:1025D00010000020ADF812000720ADF8140001A98A
:1025E000054800F06BF80121034800F04DF807B0F2
:1025F00000BD0000000801400030014000B587B078
:1026000001218803FFF7C6FE01210920FFF7D2FE52
:102610004FF46040ADF8180018208DF81B0003201F
:102620008DF81A0006A91648FEF797FC4FF4604192
:102630001348FEF71FFD0020ADF804004FF4827030
:10264000ADF806000020ADF80800ADF80A00ADF8BE
:102650000C004FF40070ADF80E001820ADF810001B
:102660000020ADF812000720ADF8140001A90548BC
:1026700000F024F80121034800F006F807B000BD7F
:10268000000C01400038004021B1028842F04002B5
:10269000028004E002884FF6BF731A400280704740
:1026A0000246002013890B400BB1012000E00020FE
:1026B00070470146888970478181704710B50022B4
:1026C000028802F441520B884C8823438C882343B0
:1026D000CC8823430C8923434C8923438C8923438F
:1026E000CC8923431A430280838B4FF2FF7423402B
:1026F00083830B8A038210BD2DE9F04106460F4605
:1027000026BB06E0601CC4B2C82C02DB0020BDE87A
:10271000F08102212048FFF7C3FF0028F2D039469C
:102720001D48FFF7C9FF002405E0601CC4B2C82C97
:1027300001DB0020EBE701211748FFF7B1FF00287C
:10274000F3D01548FFF7B5FFC5B222E005E0601CE5
:10275000C4B2C82C01DB0020D9E702210F48FFF7E3
:102760009FFF0028F3D039460C48FFF7A5FF00244F
:1027700005E0601CC4B2C82C01DB0020C7E70121C2
:102780000648FFF78DFF0028F3D00448FFF791FFBC
:10279000C5B22846BBE700000030014000380040C9
:1027A00070B505460C467DB90F4800884FF6C771D5
:1027B00008400D4908800846008820430880012110
:1027C0000A48FFF761FF0EE0084800884FF6C7711E
:1027D00008400649088008460088204308800121F7
:1027E0000248FFF751FF70BD003001400038004043
:1027F000704770B504460D4629462046FEF76EFB2D
:1028000070BD000010B586B00024142101A8FDF7AA
:10281000B2FC00BF07E00B4830F8140001A921F812
:102820001400601CC4B20A2CF5DB074800F0EAF87B
:102830000A2201A9044800F009F800F07AFC06B069
:1028400010BD000034050020000003082DE9F04110
:1028500005460F461646002400BF07E037F814105F
:102860002846FFF7C6FFAD1C601CC4B2B442F5DBBE
:10287000BDE8F08170B504460D46034A294620465E
:1028800000F028F870BD00000038014010B5044683
:102890000249204600F00EF810BD00000044004040
:1028A00010B504460249204600F02DF810BD000086
:1028B0000044004070B504460D4600BF8021284604
:1028C00000F064FB0028F9D02146284600F02BFCDC
:1028D000012070BD2DE9F04104460D46164614B99D
:1028E0000120BDE8F0810AE014F8017B314638464A
:1028F000FFF7E0FF08B90020F3E7681E85B2002D5E
:10290000F2D10120EDE770B504460E460CB9012066
:1029100070BD11E014F8015B0A2D06D131460D207F
:10292000FFF7C8FF08B90020F2E731462846FFF755
:10293000C1FF08B90020EBE720780028EAD1012088
:10294000E6E710B500F002F810BD00000CB500205D
:10295000019000902A48006840F4803028490860BF
:1029600000BF2748006800F4003000900198401C28
:102970000190009818B90198B0F5A06FF1D12048E6
:10298000006800F4003010B10120009001E0002048
:1029900000900098012831D11948406818494860D2
:1029A00008464068486008464068486008464068F5
:1029B00020F47C1048600846406840F49810486055
:1029C0000846006840F08070086000BF0C4800684E
:1029D00000F000700028F9D00948406820F003009A
:1029E000074948600846406840F00200486000BF60
:1029F0000348406800F00C000828F9D10CBD000025
:102A00000010024010B50446FEF788FA2046FEF793
:102A10001BFA10BD042808D14FF0E021096941F0EC
:102A200004014FF0E022116107E04FF0E021096955
:102A300021F004014FF0E02211617047704700005F
:102A400010B51448006840F00100124908600846BB
:102A50004068114908400F494860084600680F491E
:102A600008400C4908600846006820F4802008608F
:102A70000846406820F4FE0048604FF41F0088605C
:102A80000020C862FFF75DFF4FF000600449086056
:102A900010BD0000001002400000FFF8FFFFF6FE2E
:102AA00008ED00E010B50121204800F07EF8002874
:102AB0003AD001211D4800F069F81D480088401CEB
:102AC0001B4908801B480088401C1A4908801A4886
:102AD0000088401C1849088018480078C0B14FF49D
:102AE00000711748FEF7C6FA16480088401C1549C1
:102AF000088008460088B0F5C87F09DB4FF40071F4
:102B00000F48FEF7B5FA00200E4908800B490870FF
:102B10000948008841F28831884202D100200649E4
:102B2000088001200849087010BD00000004004022
:102B3000260000203A000020280000202C00002061
:102B4000001001402E0000202A0000203EB505465E
:102B50000C4601210220FFF71DFCADF80450ADF832
:102B600000400020ADF80600ADF8020069460648B6
:102B700000F036F801221146034800F027F8012141
:102B8000014800F006F83EBD00040040CA4302823E
:102B9000704721B1028842F00102028004E00288FD
:102BA0004FF6FE731A400280704730B5024600208F
:102BB00000230024158A05EA0103958905EA01042A
:102BC00013B10CB1012000E0002030BD1AB183899F
:102BD0000B43838102E083898B438381704700002C
:102BE000002202881D4B98420ED01D4B98420BD0FC
:102BF000B0F1804F08D01B4B984205D01A4B984239
:102C000002D01A4B984204D14FF68F731A404B886A
:102C10001A43174B984207D0164B984204D04FF6F0
:102C2000FF431A40CB881A4302808B8883850B8828
:102C300003850A4B98420BD0094B984208D00E4BA3
:102C4000984205D00D4B984202D00D4B984201D1CD
:102C50000B7A03860123838270470000002C014019
:102C6000003401400004004000080040000C004017
:102C700000100040001400400040014000440140AA
:102C80000048014010B540F22551124800F08BF980
:102C900088B140F225510F4800F0CFF80D4800F000
:102CA0003DFAC4B20C480D49097844540B480078E9
:102CB000401C0A4908700821064800F067F90128FD
:102CC00006D10821034800F0AFF8024800F026FAC8
:102CD00010BD0000003801400C010020030000205E
:102CE00010B540F22551124800F05DF988B140F26C
:102CF00025510F4800F0A1F80D4800F00FFAC4B2BA
:102D00000C480D49097844540B480078401C0A4986
:102D100008700821064800F039F9012806D1082179
:102D2000034800F081F8024800F0F8F910BD0000F7
:102D300000440040F40400208D00002010B586B04F
:102D4000044601210520FFF735FB01214804FFF768
:102D500021FB0420ADF8140003208DF81600182084
:102D60008DF8170005A91548FEF7F7F80820ADF80B
:102D7000140004208DF8170005A91048FEF7EDF89F
:102D800001940020ADF80800ADF80A00ADF80C0081
:102D9000ADF810000C20ADF80E0001A9084800F0B5
:102DA00051F9012240F22551054800F026F9012190
:102DB000034800F051F806B010BD000000080140C3
:102DC0000044004010B540F22551144800F0EBF8E3
:102DD000B0B140F22551114800F02FF80F4800F033
:102DE0009DF9C4B20E480F49097844540D48007843
:102DF000401C0C4908700846007800F00F0008706D
:102E00000821064800F0C2F8012806D1082103482D
:102E100000F00AF8014800F081F910BD00480040B8
:102E2000D40100200900002001F40072B2F5007FF7
:102E300000D100BFCA430280704710B500220023B2
:102E400040F66A14A14200D100BF0A120124944046
:102E5000A3B2DC43048010BD21B1828942F4005248
:102E6000828104E082894DF6FF731A4082817047A7
:102E700000B585B0012144F20400FFF79BFA4FF43E
:102E80000070ADF8000003208DF8020018208DF8C6
:102E9000030069463948FEF760F84FF48060ADF8EA
:102EA000000004208DF8030069463448FEF755F809
:102EB0004FF4164001900020ADF80800ADF80A006C
:102EC000ADF80C00ADF810000C20ADF80E0001A913
:102ED0002B4800F0B7F8012240F22551284800F0B5
:102EE0008CF801212648FFF7B7FF01218804FFF77E
:102EF00051FA01210820FFF75DFA4FF48060ADF828
:102F0000000003208DF8020018208DF803006946A8
:102F10001C48FEF722F84FF40060ADF800000420D2
:102F20008DF8030069461748FEF717F84FF49650DE
:102F300001900020ADF80800ADF80A00ADF80C00D3
:102F4000ADF810000C20ADF80E0001A90E4800F0FD
:102F500079F801A90C4800F075F8012240F22551DA
:102F6000094800F04AF801210748FFF775FF4021A2
:102F70000348FFF759FF05B000BD000000080140FD
:102F800000380140000C014000480040024600208B
:102F9000B1F5007F00D100BF13880B400BB10120B9
:102FA00000E00020704770B5024600240023002591
:102FB000002040F66A16B14200D100BFC1F34215AD
:102FC00001F01F03012606FA03F3012D02D19689B1
:102FD000334006E0022D02D1168A334001E0968A82
:102FE00033400C12012606FA04F41688344013B15B
:102FF0000CB1012000E0002070BDF0B503460024B4
:1030000000260025002040F66A17B94200D100BF13
:103010001846C1F3421401F01F06012707FA06F50E
:10302000012C01D10C3004E0022C01D1103000E061
:1030300014301AB107682F43076002E00768AF43F6
:103040000760F0BD2DE9F04786B005460E46002426
:10305000A24600BFA1460027B08900B100BF2F469D
:103060002C8A4CF6FF700440F08804432C82AC8913
:103070004EF6F3100440B088318908437189084343
:103080000443AC81AC8A4FF6FF400440B08904434E
:10309000AC8201A8FFF7D6F91F48874202D1DDF8BC
:1030A00010A001E0DDF80CA0A88900F4004040B1B8
:1030B0000AEBCA0000EB0A1031684900B0FBF1F8D6
:1030C00007E00AEBCA0000EB0A1031688900B0FB88
:1030D000F1F86420B8FBF0F004012009642101FB41
:1030E0001089A88900F4004040B1322000EBC900EB
:1030F000B0FBF1F000F00700044308E0322000EBE1
:1031000009106421B0FBF1F000F00F0004432C81A2
:1031100006B0BDE8F087000000380140014688880D
:10312000C0F308007047C1F308028280704700BFF7
:10313000FEE710B5FDF7C8FE10BD0000014A0249C8
:1031400000F013B8B9310008A400002002E008C85C
:10315000121F08C1002AFAD170477047002001E011
:1031600001C1121F002AFBD170472DE9F04116461C
:103170000F460446002503E03946B047641C6D1C29
:1031800020780028F8D12846BDE8F08110B5024625
:103190000BE0C82007E0122101E04B1E99B2002984
:1031A000FBDC431E98B20028F5DC131EA2F10104DB
:1031B000A2B2EED110BD000070B504460D46E0B2DB
:1031C0000549088000BF40210348001FFFF7DEFECD
:1031D0000028F8D0204670BD0438014008B5012110
:1031E0001020FFF7E7F80120ADF8000010208DF85F
:1031F000030003208DF8020069460D48FDF7ADFE7F
:1032000001210B48FDF736FF4FF40070ADF80000C8
:1032100010208DF8030003208DF802006946044851
:10322000FDF79BFE4FF400710148FDF721FF08BD3B
:1032300000100140FFF7CEF8FFF72AF840F27121A5
:103240000420FDF73BFFFDF735FF41F61F41092044
:10325000FFF77CFCFFF7C2FFFFF70AFE4FF4E130F7
:10326000FFF76CFDFDF786FFFDF724FF02E056A097
:10327000FFF764FF0120FDF751FF0028F7D1FDF7AC
:1032800027FDFDF717FF54480068C0435349C1F8B4
:103290008001C820FFF77AFF5048D0F88001C04372
:1032A0004E49C1F8800106214DA0FDF7B2FD4EA0A8
:1032B000FFF7F6FAFDF7FEFE4CA0FFF73FFF0120F7
:1032C000FEF7A6FAFFF728F951480078514908702F
:1032D00008460078172869D2DFE800F00C101418AF
:1032E0001C2024282C3034383C4044484C5054583E
:1032F0005C60640048A0FFF721FF57E049A0FFF79A
:103300001DFF53E04AA0FFF719FF4FE04BA0FFF766
:1033100015FF4BE04CA0FFF711FF47E04DA0FFF772
:103320000DFF43E04FA0FFF709FF3FE050A0FFF77C
:1033300005FF3BE052A0FFF701FF37E053A0FFF786
:10334000FDFE33E054A0FFF7F9FE2FE055A0FFF794
:10335000F5FE2BE057A0FFF7F1FE27E05AA0FFF79C
:10336000EDFE23E05CA0FFF7E9FE1FE05EA0FFF7A3
:10337000E5FE1BE060A0FFF7E1FE17E062A0FFF7AB
:10338000DDFE13E064A0FFF7D9FE0FE066A0FFF7B3
:10339000D5FE0BE068A0FFF7D1FE07E06AA0FFF7BB
:1033A000CDFE03E06BA0FFF7C9FE00BF00BF012008
:1033B0006C4908703220FFF7E9FE03E0FCF70CFFD0
:1033C000FDF774F9FAE7000054686520322E34479F
:1033D000204572726F722100800122420000224259
:1033E00031323334353600000A0000000A5043B64B
:1033F000D4C2EBC8EDBCFECDA8D3C3B0E6B1BE5677
:10340000322E342D32303139303930360A00000056
:103410004805002032000020BDADCEF7D0ADD2E986
:103420000D0A0000CCECB2A8D0ADD2E90D0A000024
:10343000D4C6C4CFD0ADD2E90D0A0000B9F3D6DDB1
:10344000D0ADD2E90D0A0000CBC4B4A8D0ADD2E90A
:103450000D0A0000C4DAC3C9B9C5D0ADD2E90D0A5E
:1034600000000000B0B2BBD5D0ADD2E90D0A00001B
:10347000C9BDCEF7F6CEC5B5D0ADD2E90D0A000074
:1034800056434F4DB2E2CAD40D0A0000C1C9C4FE72
:10349000B5E7D0C50D0A0000C1C9C4FED2C6B6AF9B
:1034A0000D0A00005470D7A8D3C3D0ADD2E90D0ADD
:1034B00000000000C4DAC3C9B9C5D2C6B6AFD0ADEA
:1034C000D2E90D0A00000000B9E3CEF7D2C6B6AFCC
:1034D000D0ADD2E90D0A0000CBC4B4A8B5E7D0C581
:1034E000D0ADD2E90D0A0000B8A3BDA8D5E6D7C675
:1034F000D0ADD2E90D0A0000CBD5D6DDC4BEC0BC2C
:10350000D0ADD2E90D0A0000D6D8C7ECD2C6B6AF0E
:10351000D0ADD2E90D0A0000C9BDCEF7D2C6B6AF14
:10352000D0ADD2E90D0A0000B8CACBE0D2C6B6AF22
:10353000D0ADD2E90D0A0000D0C5B4EFB7E1D0ADEF
:10354000D2E90D0A00000000B5C2BAA3D0ADD2E99D
:103550000D0A0000B0B2BBD5B5E7D0C5D0ADD2E9F9
:103560000D0A00002B0000203443101001344310DA
:10357000100133200D547933200D54793443101049
:103580000101101043343223ABBA013412BBAA013B
:1035900034128675014656431000346E46100134CD
:1035A00043101001862C95010136E4A7BC01421896
:1035B000BAE801341286750133200D5400862C952B
:1035C00000005A454E4B00AABB1234003412BBAA6D
:1035D000002543101200E77EE300004222B6E90016
:1035E000C013E3000083219515004115431200002C
:1035F0001036000800000020A80000004C31000830
:10360000B8360008A8000020585F00005C310008B0
:10361000000000000000000000000000D1D1E0D058
:1036200000000000D2D200000000000000000000F6
:10363000000000000000000000000000000000008A
:10364000000000000000000000000000000000007A
:103650000000000000000000000031323334353635
:1036600037383931323334353637383900000000D5
:103670000000000000000000000031323334353615
:1036800037383931323334353637383900000000B5
:10369000000000000000000000000000000000002A
:1036A00000000000010203040102030406070809E8
:0836B0000204060800000000FE
:0400000508000131BD
:00000001FF
